:020000040000FA
:02000000FE2FD1
:100F2C000330831603138E0020308500F0308600CA
:100F3C007F3081000B108B15831203130608F00011
:100F4C0004300310F00CFF3E031DA72F7008FF3A6E
:100F5C000F39F1007108F4000B10CB2F093085000C
:100F6C000130C92F0A3085000230C92F1A30850094
:100F7C000E30C92F453085008601E42F8630C12FF5
:100F8C00D630850003308600E42F7408F000F101A0
:100F9C007108003A0319D32FC62F7008003A0319B1
:100FAC00C42F013A0319B42F033A0319B82F063A88
:100FBC000319BC2F0C3A0319C02FC62F3C30F2007A
:100FCC000030F3000130F2020030031CF303F30293
:100FDC00003073020230031972020318E82F8312D7
:100FEC0003130508F03985000B18A22F6300A22FFC
:040FFC008301962FA8
:02400E0058FF59
:00000001FF
